BL51 BANKED LINKER/LOCATER V6.22.2.0                                                    04/07/2022  20:07:47  PAGE 1


BL51 BANKED LINKER/LOCATER V6.22.2.0, INVOKED BY:
C:\KEIL_V5\C51\BIN\BL51.EXE .\Objects\main.obj, .\Objects\delay.obj, .\Objects\led_num.obj TO .\Objects\MCU_1 PRINT (.\L
>> istings\MCU_1.m51)


MEMORY MODEL: LARGE


INPUT MODULES INCLUDED:
  .\Objects\main.obj (MAIN)
  .\Objects\delay.obj (DELAY)
  .\Objects\led_num.obj (LED_NUM)
  C:\KEIL_V5\C51\LIB\C51L.LIB (?C_STARTUP)
  C:\KEIL_V5\C51\LIB\C51L.LIB (?C?SLDIV)
  C:\KEIL_V5\C51\LIB\C51L.LIB (?C_INIT)
  C:\KEIL_V5\C51\LIB\C51L.LIB (?C?ULDIV)


LINK MAP OF MODULE:  .\Objects\MCU_1 (MAIN)


            TYPE    BASE      LENGTH    RELOCATION   SEGMENT NAME
            -----------------------------------------------------

            * * * * * * *   D A T A   M E M O R Y   * * * * * * *
            REG     0000H     0008H     ABSOLUTE     "REG BANK 0"
            IDATA   0008H     0001H     UNIT         ?STACK

            * * * * * * *  X D A T A   M E M O R Y  * * * * * * *
            XDATA   0000H     000CH     UNIT         ?XD?LED_NUM
            XDATA   000CH     0003H     UNIT         ?XD?HELLO_FULL_DISPLAY?LED_NUM
            XDATA   000FH     0002H     UNIT         ?XD?MAIN
            XDATA   0011H     0002H     UNIT         _XDATA_GROUP_

            * * * * * * *   C O D E   M E M O R Y   * * * * * * *
            CODE    0000H     0003H     ABSOLUTE     
            CODE    0003H     0003H     ABSOLUTE     
            CODE    0006H     00CEH     UNIT         ?C?LIB_CODE
            CODE    00D4H     00C9H     UNIT         ?PR?HELLO_DISPLAY?LED_NUM
            CODE    019DH     009DH     UNIT         ?PR?HELLO_FULL_DISPLAY?LED_NUM
            CODE    023AH     008CH     UNIT         ?C_C51STARTUP
            CODE    02C6H     0056H     UNIT         ?PR?NUM_DISPLAY?LED_NUM
            CODE    031CH     0051H     UNIT         ?PR?_GET_VAR?LED_NUM
            CODE    036DH     0049H     UNIT         ?PR?INT0?MAIN
            CODE    03B6H     0044H     UNIT         ?C?LDIV
            CODE    03FAH     0024H     UNIT         ?C_INITSEG
            CODE    041EH     001CH     UNIT         ?PR?MAIN?MAIN
            CODE    043AH     0014H     UNIT         ?PR?MOVE?MAIN
            CODE    044EH     0012H     UNIT         ?PR?NUM_PUSH?LED_NUM
            CODE    0460H     000FH     UNIT         ?PR?HELLO_PUSH?LED_NUM
            CODE    046FH     000EH     UNIT         ?PR?_DELAY?DELAY
            CODE    047DH     0007H     UNIT         ?PR?LEDFULL?LED_NUM



OVERLAY MAP OF MODULE:   .\Objects\MCU_1 (MAIN)


BL51 BANKED LINKER/LOCATER V6.22.2.0                                                  04/07/2022  20:07:47  PAGE 2


SEGMENT                                  XDATA_GROUP
  +--> CALLED SEGMENT                  START    LENGTH
------------------------------------------------------
?PR?INT0?MAIN                          -----    -----
  +--> ?PR?_DELAY?DELAY

*** NEW ROOT ***************************************************

?C_C51STARTUP                          -----    -----
  +--> ?PR?MAIN?MAIN
  +--> ?C_INITSEG

?PR?MAIN?MAIN                          -----    -----
  +--> ?PR?MOVE?MAIN
  +--> ?PR?HELLO_PUSH?LED_NUM
  +--> ?PR?HELLO_DISPLAY?LED_NUM

?PR?HELLO_DISPLAY?LED_NUM              -----    -----
  +--> ?PR?_GET_VAR?LED_NUM
  +--> ?PR?_DELAY?DELAY

?PR?_GET_VAR?LED_NUM                   0011H    0002H



SYMBOL TABLE OF MODULE:  .\Objects\MCU_1 (MAIN)

  VALUE           TYPE          NAME
  ----------------------------------

  -------         MODULE        MAIN
  C:0000H         SYMBOL        _ICE_DUMMY_
  D:0090H         PUBLIC        P1
  D:00B0H         PUBLIC        P3
  B:00A8H.7       PUBLIC        EA
  D:00A8H         PUBLIC        IE
  D:00B8H         PUBLIC        IP
  C:041EH         PUBLIC        main
  D:0098H         PUBLIC        SCON
  D:0088H         PUBLIC        TCON
  X:000FH         PUBLIC        move_flag
  C:043AH         PUBLIC        move
  B:0088H.1       PUBLIC        IE0
  B:00A8H.0       PUBLIC        EX0
  B:0088H.0       PUBLIC        IT0
  D:00C8H         PUBLIC        T2CON
  D:00D0H         PUBLIC        PSW
  X:0010H         PUBLIC        var1
  C:036DH         PUBLIC        int0
  -------         PROC          MOVE
  C:043AH         LINE#         8
  C:043AH         LINE#         9
  C:043AH         LINE#         10
  C:044BH         LINE#         11
  C:044DH         LINE#         12
  -------         ENDPROC       MOVE
  -------         PROC          INT0
BL51 BANKED LINKER/LOCATER V6.22.2.0                                                  04/07/2022  20:07:47  PAGE 3


  C:036DH         LINE#         15
  C:038AH         LINE#         17
  C:038CH         LINE#         18
  C:0393H         LINE#         19
  C:0395H         LINE#         20
  C:039BH         LINE#         21
  -------         ENDPROC       INT0
  -------         PROC          MAIN
  C:041EH         LINE#         24
  C:041EH         LINE#         25
  C:041EH         LINE#         30
  C:0420H         LINE#         31
  C:0422H         LINE#         32
  C:0424H         LINE#         34
  C:0424H         LINE#         35
  C:0424H         LINE#         36
  C:042AH         LINE#         37
  C:042AH         LINE#         38
  C:042DH         LINE#         39
  C:0430H         LINE#         41
  C:0435H         LINE#         42
  C:0435H         LINE#         44
  C:0438H         LINE#         53
  -------         ENDPROC       MAIN
  -------         ENDMOD        MAIN

  -------         MODULE        DELAY
  C:0000H         SYMBOL        _ICE_DUMMY_
  C:046FH         PUBLIC        _delay
  -------         PROC          _DELAY
  D:0006H         SYMBOL        i
  C:046FH         LINE#         3
  C:046FH         LINE#         5
  C:046FH         LINE#         6
  C:047CH         LINE#         7
  -------         ENDPROC       _DELAY
  -------         ENDMOD        DELAY

  -------         MODULE        LED_NUM
  C:0000H         SYMBOL        _ICE_DUMMY_
  D:0080H         PUBLIC        P0
  D:0090H         PUBLIC        P1
  D:00A0H         PUBLIC        P2
  D:00B0H         PUBLIC        P3
  C:019DH         PUBLIC        hello_full_display
  D:00A8H         PUBLIC        IE
  D:00B8H         PUBLIC        IP
  X:0000H         SYMBOL        count
  C:02C6H         PUBLIC        num_display
  D:0098H         PUBLIC        SCON
  D:0088H         PUBLIC        TCON
  C:0460H         PUBLIC        hello_push
  X:0002H         PUBLIC        hello_var
  X:0008H         SYMBOL        e
  D:00C8H         PUBLIC        T2CON
  X:0009H         SYMBOL        i
  C:047DH         PUBLIC        ledfull
BL51 BANKED LINKER/LOCATER V6.22.2.0                                                  04/07/2022  20:07:47  PAGE 4


  C:031CH         SYMBOL        _get_var
  C:00D4H         PUBLIC        hello_display
  C:044EH         PUBLIC        num_push
  D:00D0H         PUBLIC        PSW
  X:000BH         SYMBOL        var2
  -------         PROC          _GET_VAR
  X:0011H         SYMBOL        k
  C:031CH         LINE#         9
  C:0324H         LINE#         10
  C:0324H         LINE#         11
  C:036CH         LINE#         12
  -------         ENDPROC       _GET_VAR
  -------         PROC          HELLO_DISPLAY
  C:00D4H         LINE#         19
  C:00D4H         LINE#         20
  C:00D4H         LINE#         21
  C:00E6H         LINE#         22
  C:00E6H         LINE#         23
  C:00E9H         LINE#         24
  C:00F2H         LINE#         25
  C:00F9H         LINE#         26
  C:00FCH         LINE#         28
  C:00FFH         LINE#         29
  C:0108H         LINE#         30
  C:010FH         LINE#         31
  C:0112H         LINE#         33
  C:0115H         LINE#         34
  C:011EH         LINE#         35
  C:0125H         LINE#         36
  C:0128H         LINE#         38
  C:012BH         LINE#         39
  C:0134H         LINE#         40
  C:013BH         LINE#         41
  C:013EH         LINE#         43
  C:0141H         LINE#         44
  C:014AH         LINE#         45
  C:0151H         LINE#         46
  C:0154H         LINE#         48
  C:0157H         LINE#         49
  C:015FH         LINE#         50
  C:0166H         LINE#         51
  C:0169H         LINE#         56
  C:0169H         LINE#         57
  C:0178H         LINE#         58
  C:0178H         LINE#         59
  C:017BH         LINE#         61
  C:017BH         LINE#         62
  C:0189H         LINE#         63
  C:0198H         LINE#         64
  C:019CH         LINE#         66
  -------         ENDPROC       HELLO_DISPLAY
  -------         PROC          HELLO_PUSH
  C:0460H         LINE#         68
  C:0460H         LINE#         69
  C:0460H         LINE#         71
  C:046EH         LINE#         77
  -------         ENDPROC       HELLO_PUSH
BL51 BANKED LINKER/LOCATER V6.22.2.0                                                  04/07/2022  20:07:47  PAGE 5


  -------         PROC          NUM_DISPLAY
  C:02C6H         LINE#         79
  C:02C6H         LINE#         80
  C:02C6H         LINE#         81
  C:02D5H         LINE#         82
  C:02D5H         LINE#         84
  C:02D8H         LINE#         85
  C:02DEH         LINE#         86
  C:02E5H         LINE#         87
  C:02E8H         LINE#         92
  C:02E8H         LINE#         93
  C:02F7H         LINE#         94
  C:02F7H         LINE#         95
  C:02FAH         LINE#         96
  C:02FAH         LINE#         97
  C:0308H         LINE#         98
  C:0317H         LINE#         99
  C:031BH         LINE#         101
  -------         ENDPROC       NUM_DISPLAY
  -------         PROC          NUM_PUSH
  C:044EH         LINE#         104
  C:044EH         LINE#         105
  C:044EH         LINE#         106
  C:045FH         LINE#         107
  -------         ENDPROC       NUM_PUSH
  -------         PROC          LEDFULL
  C:047DH         LINE#         109
  C:047DH         LINE#         110
  C:047DH         LINE#         111
  C:0480H         LINE#         112
  C:0483H         LINE#         113
  -------         ENDPROC       LEDFULL
  -------         PROC          HELLO_FULL_DISPLAY
  -------         DO            
  X:000CH         SYMBOL        var3
  X:000DH         SYMBOL        j
  -------         ENDDO         
  C:019DH         LINE#         116
  C:019DH         LINE#         117
  C:019DH         LINE#         118
  C:01ACH         LINE#         119
  C:01ACH         LINE#         120
  C:01B2H         LINE#         122
  C:01B7H         LINE#         123
  C:01B7H         LINE#         124
  C:01C8H         LINE#         125
  C:01CAH         LINE#         126
  C:01DDH         LINE#         127
  C:01E4H         LINE#         128
  C:01E7H         LINE#         129
  C:0206H         LINE#         134
  C:0206H         LINE#         135
  C:0215H         LINE#         136
  C:0215H         LINE#         137
  C:0218H         LINE#         139
  C:0218H         LINE#         140
  C:0226H         LINE#         141
BL51 BANKED LINKER/LOCATER V6.22.2.0                                                  04/07/2022  20:07:47  PAGE 6


  C:0235H         LINE#         142
  C:0239H         LINE#         144
  -------         ENDPROC       HELLO_FULL_DISPLAY
  -------         ENDMOD        LED_NUM

  -------         MODULE        ?C?SLDIV
  C:03B6H         PUBLIC        ?C?SLDIV
  -------         ENDMOD        ?C?SLDIV

  -------         MODULE        ?C?ULDIV
  C:0042H         PUBLIC        ?C?ULDIV
  -------         ENDMOD        ?C?ULDIV

*** WARNING L16: UNCALLED SEGMENT, IGNORED FOR OVERLAY PROCESS
    SEGMENT: ?PR?NUM_DISPLAY?LED_NUM

*** WARNING L16: UNCALLED SEGMENT, IGNORED FOR OVERLAY PROCESS
    SEGMENT: ?PR?NUM_PUSH?LED_NUM

*** WARNING L16: UNCALLED SEGMENT, IGNORED FOR OVERLAY PROCESS
    SEGMENT: ?PR?LEDFULL?LED_NUM

*** WARNING L16: UNCALLED SEGMENT, IGNORED FOR OVERLAY PROCESS
    SEGMENT: ?PR?HELLO_FULL_DISPLAY?LED_NUM

Program Size: data=9.0 xdata=19 code=1156
LINK/LOCATE RUN COMPLETE.  4 WARNING(S),  0 ERROR(S)
